C51 COMPILER V9.51   SPIM_INT                                                              10/14/2013 23:29:43 PAGE 1   


C51 COMPILER V9.51, COMPILATION OF MODULE SPIM_INT
OBJECT MODULE PLACED IN .\DP8051_Keil_951\Debug\SPIM_INT.obj
COMPILER INVOKED BY: C:\Program Files (x86)\Cypress\PSoC Creator\3.0\PSoC Creator\import\keil\pk51\9.51\C51\BIN\c51.exe 
                    -.\Generated_Source\PSoC3\SPIM_INT.c NOIV LARGE MODDP2 OMF2 VB(1) PR(.\DP8051_Keil_951\Debug\SPIM_INT.lst) CD DB NOIP OT(
                    -5,SIZE) INCDIR(.,.\Generated_Source\PSoC3) OJ(.\DP8051_Keil_951\Debug\SPIM_INT.obj)

line level    source

   1          /*******************************************************************************
   2          * File Name: SPIM_INT.c
   3          * Version 2.40
   4          *
   5          * Description:
   6          *  This file provides all Interrupt Service Routine (ISR) for the SPI Master
   7          *  component.
   8          *
   9          * Note:
  10          *  None.
  11          *
  12          ********************************************************************************
  13          * Copyright 2008-2012, Cypress Semiconductor Corporation.  All rights reserved.
  14          * You may use this file only in accordance with the license, terms, conditions,
  15          * disclaimers, and limitations in the end user license agreement accompanying
  16          * the software package with which this file was provided.
  17          *******************************************************************************/
  18          
  19          #include "SPIM_PVT.h"
  20          
  21          /* User code required at start of ISR */
  22          /* `#START SPIM_ISR_START_DEF` */
  23          
  24          /* `#END` */
  25          
  26          
  27          /*******************************************************************************
  28          * Function Name: SPIM_TX_ISR
  29          ********************************************************************************
  30          *
  31          * Summary:
  32          *  Interrupt Service Routine for TX portion of the SPI Master.
  33          *
  34          * Parameters:
  35          *  None.
  36          *
  37          * Return:
  38          *  None.
  39          *
  40          * Global variables:
  41          *  SPIM_txBufferWrite - used for the account of the bytes which
  42          *  have been written down in the TX software buffer.
  43          *  SPIM_txBufferRead - used for the account of the bytes which
  44          *  have been read from the TX software buffer, modified when exist data to
  45          *  sending and FIFO Not Full.
  46          *  SPIM_txBuffer[SPIM_TX_BUFFER_SIZE] - used to store
  47          *  data to sending.
  48          *  All described above Global variables are used when Software Buffer is used.
  49          *
  50          *******************************************************************************/
  51          CY_ISR(SPIM_TX_ISR)
  52          {
  53   1          #if(SPIM_TX_SOFTWARE_BUF_ENABLED)
C51 COMPILER V9.51   SPIM_INT                                                              10/14/2013 23:29:43 PAGE 2   

  54   1              uint8 tmpStatus;
  55   1          #endif /* (SPIM_TX_SOFTWARE_BUF_ENABLED) */
  56   1      
  57   1          /* User code required at start of ISR */
  58   1          /* `#START SPIM_TX_ISR_START` */
  59   1      
  60   1          /* `#END` */
  61   1      
  62   1          #if(SPIM_TX_SOFTWARE_BUF_ENABLED)
  63   1              /* Check if TX data buffer is not empty and there is space in TX FIFO */
  64   1              while(SPIM_txBufferRead != SPIM_txBufferWrite)
  65   1              {
  66   2                  tmpStatus = SPIM_GET_STATUS_TX(SPIM_swStatusTx);
  67   2                  SPIM_swStatusTx = tmpStatus;
  68   2      
  69   2                  if(0u != (SPIM_swStatusTx & SPIM_STS_TX_FIFO_NOT_FULL))
  70   2                  {
  71   3                      if(0u == SPIM_txBufferFull)
  72   3                      {
  73   4                         SPIM_txBufferRead++;
  74   4      
  75   4                          if(SPIM_txBufferRead >= SPIM_TX_BUFFER_SIZE)
  76   4                          {
  77   5                              SPIM_txBufferRead = 0u;
  78   5                          }
  79   4                      }
  80   3                      else
  81   3                      {
  82   4                          SPIM_txBufferFull = 0u;
  83   4                      }
  84   3      
  85   3                      /* Move data from the Buffer to the FIFO */
  86   3                      CY_SET_REG8(SPIM_TXDATA_PTR,
  87   3                          SPIM_txBuffer[SPIM_txBufferRead]);
  88   3                  }
  89   2                  else
  90   2                  {
  91   3                      break;
  92   3                  }
  93   2              }
  94   1      
  95   1              if(SPIM_txBufferRead == SPIM_txBufferWrite)
  96   1              {
  97   2                  /* TX Buffer is EMPTY: disable interrupt on TX NOT FULL */
  98   2                  SPIM_TX_STATUS_MASK_REG &= ((uint8) ~SPIM_STS_TX_FIFO_NOT_FULL);
  99   2              }
 100   1      
 101   1          #endif /* (SPIM_TX_SOFTWARE_BUF_ENABLED) */
 102   1      
 103   1          /* User code required at end of ISR (Optional) */
 104   1          /* `#START SPIM_TX_ISR_END` */
 105   1      
 106   1          /* `#END` */
 107   1      }
 108          
 109          
 110          /*******************************************************************************
 111          * Function Name: SPIM_RX_ISR
 112          ********************************************************************************
 113          *
 114          * Summary:
 115          *  Interrupt Service Routine for RX portion of the SPI Master.
C51 COMPILER V9.51   SPIM_INT                                                              10/14/2013 23:29:43 PAGE 3   

 116          *
 117          * Parameters:
 118          *  None.
 119          *
 120          * Return:
 121          *  None.
 122          *
 123          * Global variables:
 124          *  SPIM_rxBufferWrite - used for the account of the bytes which
 125          *  have been written down in the RX software buffer modified when FIFO contains
 126          *  new data.
 127          *  SPIM_rxBufferRead - used for the account of the bytes which
 128          *  have been read from the RX software buffer, modified when overflow occurred.
 129          *  SPIM_rxBuffer[SPIM_RX_BUFFER_SIZE] - used to store
 130          *  received data, modified when FIFO contains new data.
 131          *  All described above Global variables are used when Software Buffer is used.
 132          *
 133          *******************************************************************************/
 134          CY_ISR(SPIM_RX_ISR)
 135          {
 136   1          #if(SPIM_RX_SOFTWARE_BUF_ENABLED)
 137   1              uint8 tmpStatus;
 138   1              uint8 rxData;
 139   1          #endif /* (SPIM_RX_SOFTWARE_BUF_ENABLED) */
 140   1      
 141   1          /* User code required at start of ISR */
 142   1          /* `#START SPIM_RX_ISR_START` */
 143   1      
 144   1          /* `#END` */
 145   1      
 146   1          #if(SPIM_RX_SOFTWARE_BUF_ENABLED)
 147   1      
 148   1              tmpStatus = SPIM_GET_STATUS_RX(SPIM_swStatusRx);
 149   1              SPIM_swStatusRx = tmpStatus;
 150   1      
 151   1              /* Check if RX data FIFO has some data to be moved into the RX Buffer */
 152   1              while(0u != (SPIM_swStatusRx & SPIM_STS_RX_FIFO_NOT_EMPTY))
 153   1              {
 154   2                  rxData = CY_GET_REG8(SPIM_RXDATA_PTR);
 155   2      
 156   2                  /* Set next pointer. */
 157   2                  SPIM_rxBufferWrite++;
 158   2                  if(SPIM_rxBufferWrite >= SPIM_RX_BUFFER_SIZE)
 159   2                  {
 160   3                      SPIM_rxBufferWrite = 0u;
 161   3                  }
 162   2      
 163   2                  if(SPIM_rxBufferWrite == SPIM_rxBufferRead)
 164   2                  {
 165   3                      SPIM_rxBufferRead++;
 166   3                      if(SPIM_rxBufferRead >= SPIM_RX_BUFFER_SIZE)
 167   3                      {
 168   4                          SPIM_rxBufferRead = 0u;
 169   4                      }
 170   3      
 171   3                      SPIM_rxBufferFull = 1u;
 172   3                  }
 173   2      
 174   2                  /* Move data from the FIFO to the Buffer */
 175   2                  SPIM_rxBuffer[SPIM_rxBufferWrite] = rxData;
 176   2      
 177   2                  tmpStatus = SPIM_GET_STATUS_RX(SPIM_swStatusRx);
C51 COMPILER V9.51   SPIM_INT                                                              10/14/2013 23:29:43 PAGE 4   

 178   2                  SPIM_swStatusRx = tmpStatus;
 179   2              }
 180   1      
 181   1          #endif /* (SPIM_RX_SOFTWARE_BUF_ENABLED) */
 182   1      
 183   1          /* User code required at end of ISR (Optional) */
 184   1          /* `#START SPIM_RX_ISR_END` */
 185   1      
 186   1          /* `#END` */
 187   1      }
 188          
 189          /* [] END OF FILE */
C51 COMPILER V9.51   SPIM_INT                                                              10/14/2013 23:29:43 PAGE 5   

ASSEMBLY LISTING OF GENERATED OBJECT CODE


             ; FUNCTION SPIM_TX_ISR (BEGIN)
0000 C0E0              PUSH    ACC
0002 C083              PUSH    DPH
0004 C082              PUSH    DPL
0006 C085              PUSH    DPH1
0008 C084              PUSH    DPL1
000A C086              PUSH    DPS
000C 758600            MOV     DPS,#00H
000F C000        E     PUSH    ?C?XPAGE1SFR
0011 750000      E     MOV     ?C?XPAGE1SFR,#?C?XPAGE1RST
0014 C0D0              PUSH    PSW
0016 75D000            MOV     PSW,#00H
0019 C007              PUSH    AR7
                                           ; SOURCE LINE # 51
001B         ?C0001:
                                           ; SOURCE LINE # 64
001B 900000      E     MOV     DPTR,#SPIM_txBufferWrite
001E E0                MOVX    A,@DPTR
001F FF                MOV     R7,A
0020 900000      E     MOV     DPTR,#SPIM_txBufferRead
0023 E0                MOVX    A,@DPTR
0024 6F                XRL     A,R7
0025 6046              JZ      ?C0002
                                           ; SOURCE LINE # 65
                                           ; SOURCE LINE # 66
0027 900000      E     MOV     DPTR,#SPIM_swStatusTx
002A E0                MOVX    A,@DPTR
002B 5409              ANL     A,#09H
002D FF                MOV     R7,A
002E 906467            MOV     DPTR,#06467H
0031 E0                MOVX    A,@DPTR
0032 4F                ORL     A,R7
0033 FF                MOV     R7,A
;---- Variable 'tmpStatus' assigned to Register 'R7' ----
                                           ; SOURCE LINE # 67
0034 900000      E     MOV     DPTR,#SPIM_swStatusTx
0037 F0                MOVX    @DPTR,A
                                           ; SOURCE LINE # 69
0038 E0                MOVX    A,@DPTR
0039 30E231            JNB     ACC.2,?C0002
                                           ; SOURCE LINE # 70
                                           ; SOURCE LINE # 71
003C 900000      E     MOV     DPTR,#SPIM_txBufferFull
003F E0                MOVX    A,@DPTR
0040 7010              JNZ     ?C0004
                                           ; SOURCE LINE # 72
                                           ; SOURCE LINE # 73
0042 900000      E     MOV     DPTR,#SPIM_txBufferRead
0045 E0                MOVX    A,@DPTR
0046 04                INC     A
0047 F0                MOVX    @DPTR,A
                                           ; SOURCE LINE # 75
0048 E0                MOVX    A,@DPTR
0049 C3                CLR     C
004A 9408              SUBB    A,#08H
004C 4009              JC      ?C0006
                                           ; SOURCE LINE # 76
                                           ; SOURCE LINE # 77
004E E4                CLR     A
C51 COMPILER V9.51   SPIM_INT                                                              10/14/2013 23:29:43 PAGE 6   

004F F0                MOVX    @DPTR,A
                                           ; SOURCE LINE # 78
                                           ; SOURCE LINE # 79
0050 8005              SJMP    ?C0006
0052         ?C0004:
                                           ; SOURCE LINE # 81
                                           ; SOURCE LINE # 82
0052 900000      E     MOV     DPTR,#SPIM_txBufferFull
0055 E4                CLR     A
0056 F0                MOVX    @DPTR,A
                                           ; SOURCE LINE # 83
0057         ?C0006:
                                           ; SOURCE LINE # 87
0057 900000      E     MOV     DPTR,#SPIM_txBufferRead
005A E0                MOVX    A,@DPTR
005B 2400        E     ADD     A,#LOW SPIM_txBuffer
005D F582              MOV     DPL,A
005F E4                CLR     A
0060 3400        E     ADDC    A,#HIGH SPIM_txBuffer
0062 F583              MOV     DPH,A
0064 E0                MOVX    A,@DPTR
0065 906547            MOV     DPTR,#06547H
0068 F0                MOVX    @DPTR,A
                                           ; SOURCE LINE # 88
0069 80B0              SJMP    ?C0001
                                           ; SOURCE LINE # 90
                                           ; SOURCE LINE # 91
                                           ; SOURCE LINE # 92
                                           ; SOURCE LINE # 93
006B 80AE              SJMP    ?C0001
006D         ?C0002:
                                           ; SOURCE LINE # 95
006D 900000      E     MOV     DPTR,#SPIM_txBufferWrite
0070 E0                MOVX    A,@DPTR
0071 FF                MOV     R7,A
0072 900000      E     MOV     DPTR,#SPIM_txBufferRead
0075 E0                MOVX    A,@DPTR
0076 B50707            CJNE    A,AR7,?C0009
                                           ; SOURCE LINE # 96
                                           ; SOURCE LINE # 98
0079 906487            MOV     DPTR,#06487H
007C E0                MOVX    A,@DPTR
007D 54FB              ANL     A,#0FBH
007F F0                MOVX    @DPTR,A
                                           ; SOURCE LINE # 99
                                           ; SOURCE LINE # 107
0080         ?C0009:
0080 D007              POP     AR7
0082 D0D0              POP     PSW
0084 D000        E     POP     ?C?XPAGE1SFR
0086 D086              POP     DPS
0088 D084              POP     DPL1
008A D085              POP     DPH1
008C D082              POP     DPL
008E D083              POP     DPH
0090 D0E0              POP     ACC
0092 32                RETI    
             ; FUNCTION SPIM_TX_ISR (END)

             ; FUNCTION SPIM_RX_ISR (BEGIN)
0000 C0E0              PUSH    ACC
0002 C083              PUSH    DPH
C51 COMPILER V9.51   SPIM_INT                                                              10/14/2013 23:29:43 PAGE 7   

0004 C082              PUSH    DPL
0006 C085              PUSH    DPH1
0008 C084              PUSH    DPL1
000A C086              PUSH    DPS
000C 758600            MOV     DPS,#00H
000F C000        E     PUSH    ?C?XPAGE1SFR
0011 750000      E     MOV     ?C?XPAGE1SFR,#?C?XPAGE1RST
0014 C0D0              PUSH    PSW
0016 75D000            MOV     PSW,#00H
0019 C005              PUSH    AR5
001B C006              PUSH    AR6
001D C007              PUSH    AR7
                                           ; SOURCE LINE # 134
;---- Variable 'rxData' assigned to Register 'R7' ----
                                           ; SOURCE LINE # 148
001F 900000      E     MOV     DPTR,#SPIM_swStatusRx
0022 E0                MOVX    A,@DPTR
0023 5440              ANL     A,#040H
0025 FE                MOV     R6,A
0026 906564            MOV     DPTR,#06564H
0029 E0                MOVX    A,@DPTR
002A 4E                ORL     A,R6
002B FE                MOV     R6,A
;---- Variable 'tmpStatus' assigned to Register 'R6' ----
                                           ; SOURCE LINE # 149
002C 900000      E     MOV     DPTR,#SPIM_swStatusRx
002F F0                MOVX    @DPTR,A
0030         ?C0010:
                                           ; SOURCE LINE # 152
0030 900000      E     MOV     DPTR,#SPIM_swStatusRx
0033 E0                MOVX    A,@DPTR
0034 30E555            JNB     ACC.5,?C0015
                                           ; SOURCE LINE # 153
                                           ; SOURCE LINE # 154
0037 906557            MOV     DPTR,#06557H
003A E0                MOVX    A,@DPTR
003B FF                MOV     R7,A
                                           ; SOURCE LINE # 157
003C 900000      E     MOV     DPTR,#SPIM_rxBufferWrite
003F E0                MOVX    A,@DPTR
0040 04                INC     A
0041 F0                MOVX    @DPTR,A
                                           ; SOURCE LINE # 158
0042 E0                MOVX    A,@DPTR
0043 C3                CLR     C
0044 9408              SUBB    A,#08H
0046 4002              JC      ?C0012
                                           ; SOURCE LINE # 159
                                           ; SOURCE LINE # 160
0048 E4                CLR     A
0049 F0                MOVX    @DPTR,A
                                           ; SOURCE LINE # 161
004A         ?C0012:
                                           ; SOURCE LINE # 163
004A 900000      E     MOV     DPTR,#SPIM_rxBufferRead
004D E0                MOVX    A,@DPTR
004E FD                MOV     R5,A
004F 900000      E     MOV     DPTR,#SPIM_rxBufferWrite
0052 E0                MOVX    A,@DPTR
0053 B50514            CJNE    A,AR5,?C0013
                                           ; SOURCE LINE # 164
                                           ; SOURCE LINE # 165
C51 COMPILER V9.51   SPIM_INT                                                              10/14/2013 23:29:43 PAGE 8   

0056 900000      E     MOV     DPTR,#SPIM_rxBufferRead
0059 E0                MOVX    A,@DPTR
005A 04                INC     A
005B F0                MOVX    @DPTR,A
                                           ; SOURCE LINE # 166
005C E0                MOVX    A,@DPTR
005D C3                CLR     C
005E 9408              SUBB    A,#08H
0060 4002              JC      ?C0014
                                           ; SOURCE LINE # 167
                                           ; SOURCE LINE # 168
0062 E4                CLR     A
0063 F0                MOVX    @DPTR,A
                                           ; SOURCE LINE # 169
0064         ?C0014:
                                           ; SOURCE LINE # 171
0064 900000      E     MOV     DPTR,#SPIM_rxBufferFull
0067 7401              MOV     A,#01H
0069 F0                MOVX    @DPTR,A
                                           ; SOURCE LINE # 172
006A         ?C0013:
                                           ; SOURCE LINE # 175
006A 900000      E     MOV     DPTR,#SPIM_rxBufferWrite
006D E0                MOVX    A,@DPTR
006E 2400        E     ADD     A,#LOW SPIM_rxBuffer
0070 F582              MOV     DPL,A
0072 E4                CLR     A
0073 3400        E     ADDC    A,#HIGH SPIM_rxBuffer
0075 F583              MOV     DPH,A
0077 EF                MOV     A,R7
0078 F0                MOVX    @DPTR,A
                                           ; SOURCE LINE # 177
0079 900000      E     MOV     DPTR,#SPIM_swStatusRx
007C E0                MOVX    A,@DPTR
007D 5440              ANL     A,#040H
007F FD                MOV     R5,A
0080 906564            MOV     DPTR,#06564H
0083 E0                MOVX    A,@DPTR
0084 4D                ORL     A,R5
0085 FE                MOV     R6,A
                                           ; SOURCE LINE # 178
0086 900000      E     MOV     DPTR,#SPIM_swStatusRx
0089 F0                MOVX    @DPTR,A
                                           ; SOURCE LINE # 179
008A 80A4              SJMP    ?C0010
                                           ; SOURCE LINE # 187
008C         ?C0015:
008C D007              POP     AR7
008E D006              POP     AR6
0090 D005              POP     AR5
0092 D0D0              POP     PSW
0094 D000        E     POP     ?C?XPAGE1SFR
0096 D086              POP     DPS
0098 D084              POP     DPL1
009A D085              POP     DPH1
009C D082              POP     DPL
009E D083              POP     DPH
00A0 D0E0              POP     ACC
00A2 32                RETI    
             ; FUNCTION SPIM_RX_ISR (END)


C51 COMPILER V9.51   SPIM_INT                                                              10/14/2013 23:29:43 PAGE 9   


MODULE INFORMATION:   STATIC OVERLAYABLE
   CODE SIZE        =    310    ----
   CONSTANT SIZE    =   ----    ----
   XDATA SIZE       =   ----    ----
   PDATA SIZE       =   ----    ----
   DATA SIZE        =   ----    ----
   IDATA SIZE       =   ----    ----
   BIT SIZE         =   ----    ----
   EDATA SIZE       =   ----    ----
   HDATA SIZE       =   ----    ----
   XDATA CONST SIZE =   ----    ----
   FAR CONST SIZE   =   ----    ----
END OF MODULE INFORMATION.


C51 COMPILATION COMPLETE.  0 WARNING(S),  0 ERROR(S)
